:107000000C945D380C9495380C947A380C947A383A
:107010000C947A380C947A380C947A380C947A3828
:107020000C947A380C947A380C947A380C947A3818
:107030000C947A380C947A380C947A380C947A3808
:107040000C947A380C947A380C947A380C947A38F8
:107050000C947A380C947A380C947A380C947A38E8
:107060000C947A380C947A38040309041C037700D2
:10707000770077002E0066006900730063006800E7
:107080006C002E00640065000E03550053004200A2
:1070900061007300700012011001FF000008C016AB
:1070A000DC05020101020001090212000101008059
:1070B000FA09040000000000000011241FBECFEFF9
:1070C000D8E0DEBFCDBF11E0A0E0B1E0ECE0F8E732
:1070D00002C005900D92A630B107D9F711E0A6E0E5
:1070E000B1E001C01D92AD33B107E1F70E94AD39A7
:1070F0000C94043C0C940038A82FB92F80E090E049
:1071000041E050EA609530E009C02D9182279795C3
:10711000879510F084279527305EC8F36F5FA8F33A
:107120000895EADF8D939D930895CF93CFB7CF93C2
:10713000DF93C3954F9BE9F74F9B11C04F9B0FC047
:107140004F9B0DC04F9B0BC04F9B09C04F9B07C06F
:107150004F9B05C04F9B03C04F9B01C081C06F93E5
:10716000C0912001DD27C95DDE4F2F9320E400C0D0
:1071700065E04F9B03C02F916F91DECF0F931F935C
:107180004F9345E55F9355E53F933BE014E009B12C
:1071900004782EC06A95C9F03150D8F109B104784D
:1071A00001130BC008942795299320E4555500F44A
:1071B0006A9569F701E069B10BC0102F66E026956A
:1071C000299320E4555518F3E2CF0FEF69B1000081
:1071D000162F455500F0404066E014780030E2F28A
:1071E00021F0000009B1047803C009B10478A9F0C6
:1071F000011309C00894279568F200C06A95A9F7A1
:1072000000E069B1E5CF102F66E0269528F2000076
:10721000ECCF11E01CBB002717C03B503195C31BBE
:10722000D04011E01CBB0881033CF9F00B34E9F0BD
:1072300020911E011981110F1213EDCF093651F162
:107240000D3211F0013E39F7009325013F915F9116
:107250004F911F910F912F916F91CCB3C0FD69CFCA
:10726000DF91CF91CFBFCF91189520912501222397
:1072700069F310912301112329F534302AF1309359
:10728000230120931F01109120013BE0311B30931B
:1072900020011AC0009123010130A4F40AE53091C5
:1072A000000134FD12C000930001C3E1D1E011C020
:1072B000052710E000C00BB919C0052710E0221FF8
:1072C00000C01DC04AE502C032ED432FC4E1D0E04A
:1072D00032E01AB114685F9A0BB11AB954E820E889
:1072E00069E420FF05270BB92795179500C000001A
:1072F0001C3FF0F66695A8F7A1F720FF05270BB90C
:107300002795179500001C3FC0F629913A9541F743
:107310000B7710912401110F0BB9C651D04011F019
:1073200010931E0111E01CBB00681AB11B77402F9F
:107330004B7755E05A95F1F70BB91AB94BB986CF8F
:107340001BB8F8941DBA1092690081E085BF15BE84
:10735000E0911101F091120109952F923F924F9205
:107360005F926F927F928F929F92AF92BF92CF92D5
:10737000DF92EF92FF920F931F93CF93DF9388E1F9
:107380000FB6F89480936000109260000FBE5F9A71
:1073900004B601FE21C214BE81E085BF82E085BF34
:1073A0004F991AC280916900836080936900E89ABE
:1073B0004F9BFECF57987894E8E86E2EE0E77E2E3C
:1073C0007CE6472E70E7572E68E6262E60E7362EBD
:1073D00058EAC52E50E7D52E46E9A42E40E7B42E34
:1073E00037E0832E31E0932E90912301935097FD47
:1073F00060C1809120012CE0E22EF12CE81AF10806
:1074000027E231E0E20EF31E80911F018D3209F078
:10741000D9C0983009F04BC133EC309313018AE5A1
:107420008093000110920B01D7013C91832F80764D
:1074300011962C911197882309F452C09092220141
:1074400080922101233009F513969C91139714968D
:107450008C91149712962C91203339F48370E82F75
:10746000F0E0EE5FFE4F80810CC0203A19F40E94DC
:10747000EE3B07C0203C21F4F70165810E94F63BFA
:1074800080E080930A0194E08AC0253011F491E0F5
:1074900086C0822F84508630E0F4D70112968D91F9
:1074A0009C91139790930D0180930C01293009F45E
:1074B00075C016969C91169790930E0115968C9117
:1074C000827080930F012093100137FD6EC02FEF63
:1074D0006DC0223009F062C0B1E0B09306015EC019
:1074E000F701828110921C01222331F410921D01B8
:1074F0002CE131E092E04DC0253019F48093240155
:1075000045C0263099F5D70113968C91813029F426
:10751000B0922201A092210106C0823031F4D092B3
:107520002201C092210192E11DC08330D1F4F70104
:107530008281882331F4309222012092210194E04B
:1075400011C0813031F450922201409221019CE11E
:1075500009C0823031F470922201609221019EE0D4
:1075600001C090E0F0E4F0930B0119C0283019F449
:1075700026E231E009C0293019F48093260106C0C3
:107580002A3021F42CE131E091E003C02CE131E01C
:1075900090E0309322012093210101C090E0D701B7
:1075A00017968C91882331F009C0292F80E88093A9
:1075B0000B0105C0F7012681291708F0292F209318
:1075C000010175C080910B0187FF71C080910E0190
:1075D000192F891708F4182F811B80930E0100E0E2
:1075E000882309F401E080911001873010F0E70151
:1075F00015C050910F01E0910C01F0910D0140E098
:107600004BC080910C0190910D01019690930D015A
:1076100080930C01019769910E94F63B9E012E19FF
:10762000211778F340C0CF018F779070892B49F4F0
:10763000F89433E030935700E895789407B600FC4F
:10764000FDCF4E5FF894D7018D919D917D01B1E002
:107650000C01B0935700E895112478949F012E5F98
:107660003F4FC9018F779070892B31F0002399F03B
:10767000411788F0552379F0F89485E080935700FE
:10768000E895789407B600FCFDCFF89491E19093CB
:107690005700E8957894F901411708F4C4CFF093A6
:1076A0000D01E0930C01002311F0109201011092E2
:1076B00023018091000184FF80C0809101018F3FF0
:1076C00009F47BC0182F893008F018E0811B8093E3
:1076D00001018091130198E88927809313011123F8
:1076E00009F458C080910B0187FF2BC080910E01D7
:1076F000811708F4182F811B80930E01009110014F
:10770000C4E1D1E0E12EFF24EC0EFD1E16C0E09195
:107710000C01F0910D01073020F0CF010E94EE3BEB
:1077200001C084918883219680910C0190910D0174
:10773000019690930D0180930C01CE15DF0539F76A
:1077400027C0209121013091220186FF0DC0A4E1C4
:10775000B1E080E090E0F901E80FF91FE491ED93CA
:1077600001961817C1F708C0D901912FE4E1F1E0A3
:107770008D9181939150E1F71150812F90E01F5F1F
:107780000196820F931F909322018093210102C0E2
:10779000193068F484E191E0612F0E949138612FE3
:1077A0006C5F6C3041F08FEF8093010104C08FEF6C
:1077B000809301016EE16093000194E189B18478C6
:1077C00031F49150D9F71092240110921E0180914A
:1077D0000601882309F408CE0E94A039F999FECF4A
:1077E00092BD81BDF89A992780B50895262FF99901
:1077F000FECF1FBA92BD81BD20BD0FB6F894FA9A94
:0C780000F99A0FBE01960895F894FFCF8E
:06780C005AFF1E950F005B
:040000030000700089
:00000001FF
